:020000021000EC
:10FC000001C0D8C0112484B790E89093610010928D
:10FC10006100882369F0982F9A70923049F081FF33
:10FC200002C097EF94BF282E80E0E7D00C9400002C
:10FC300085E08093810082E08093C80088E1809312
:10FC4000C90080E18093CC0086E08093CA008EE0FA
:10FC5000D4D0259A84E020E33CEF91E030938500F6
:10FC60002093840096BBB09BFECF1D9AA89540912F
:10FC7000C80047FD02C0815089F7B3D0813479F4C0
:10FC8000B0D0C82FC0D0C23811F480E004C088E0E2
:10FC9000C13809F083E09ED080E19CD0EECF823461
:10FCA00019F484E1B8D0F8CF853411F485E0FACFA7
:10FCB000853581F496D0082F94D0182F87FF07C080
:10FCC0008BB781608BBF000F111F9DD0E5CF8BB725
:10FCD0008E7FF8CF863579F484D08D3451F481D07D
:10FCE000CBB77FD0C170880F8C2B8BBF81E093D0B6
:10FCF000CCCF83E0FCCF843609F03AC072D0C82F55
:10FD0000D0E0DC2FCC276DD0C82B6BD0D82E5E0175
:10FD10008EEFB81AE12C32E0F32E4701EFEF8E1A86
:10FD20009E0A5FD0F701808374018A149B04A9F7AF
:10FD30006AD0F5E4DF1201C0FFCF50E040E063E09D
:10FD4000C80138D07801C12C92E0D92EF60141913A
:10FD500051916F0161E0C7012DD0F2E0EF0EF11C6F
:10FD60002297A1F750E040E065E0C80123D094CF8E
:10FD7000843789F436D0C82FD0E0DC2FCC2731D09F
:10FD8000C82B2FD040D07801F70187917F0122D076
:10FD90002197D1F781CF853739F435D08EE11AD04C
:10FDA00087E918D084E077CF813509F08ECF88E0DD
:10FDB00024D08BCFFC010A0167BFE895112407B658
:10FDC00000FCFDCF667029F0452B19F481E187BF57
:10FDD000E89508959091C80095FFFCCF8093CE00E0
:10FDE00008958091C80087FFFCCF8091C80084FDF2
:10FDF00001C0A8958091CE000895E0E6F0E098E17A
:10FE0000908380830895EDDF803219F088E0F5DF7C
:10FE1000FFCF84E1DFCFCF93C82FE3DFC150E9F7F5
:04FE2000CF91F1CFBE
:02FFFE000008F9
:040000031000FC00ED
:00000001FF
